:03000000021B835D
:0C1B830078FFE4F6D8FD7581D50200362D
:0100190022C4
:06188B008B318A32893323
:101891007571027F481219F7121BCFEF20E0F9ABE7
:1018A10031AA32A9331205477879E6FE08E6FDED43
:0118B100FF37
:0118B2002213
:100F7A0043525354005341564500434647002D3EC1
:100F8A0053320052415445434C5220554E49544223
:100F9A004C4E4B545249475452455653545254534B
:100FAA00544F505A45524F44464C54534156455259
:100FBA00535420535720202E3235203173202032AB
:100FCA007320203573202031307320333073203161
:100FDA006D2020326D2020356D202031306D203378
:100FEA00306D2031682020326820203468202000AB
:100FFA000000010004000800140028007800F00135
:10100A00E004B009601C2038407080E10046656544
:10101A0074596172644D6574724F6666204F6E2012
:10102A00204E6F2020596573204F66662054696DE3
:10103A0065416C7420547269674F66662054696D05
:10104A0065416C74204F66662054726967507772E6
:05105A00205265632037
:1018D90025E024F9F582E4340FF583220533E53355
:1018E900C394022208F608F608F62275F004A42427
:0518F90023F974102228
:10142700789976AB0876CD087600087604E408F656
:1014370008760108F60876FA0876401218ED08F6DD
:1014470078A7F608760A08F608763C08F6087614B0
:1014570008F608760F1218ED7BFF7A0F797A1217C4
:09146700D27F051217340218357A
:101A120075751D7576C012153D789AE664CD700411
:091A220018E664AB6003121427FE
:011A2B002298
:0D1B4B00C2AF7DC07C1DE4FF121AB5D2AF01
:011B5800226A
:10153D00753EFF85753F8576407541007542007596
:10154D004399E4FFAB3EAA3FA9408F8275830012F9
:10155D00051AAB41AA42A9438F8275830012055922
:10156D000FBF1AE078B2E6FFF46003EF700478B2B3
:02157D007601F5
:01157F002249
:101835007D01E4FF1219827BFF7A0F797F1217D29F
:10184500121B4BC2AF7F997B1A7DC07C1D121ABF3C
:0D185500D2AF7F02121734E4FDFF021982AA
:10097A00E4F5317BFF7A0F79841217D27F051217BB
:10098A0034A297829650FAA2969217A2979218E5E5
:10099A003175F004A4248DF9740F35F0FA7BFF1237
:1009AA0017D27F05121734853132E4F5337BFF7A8B
:1009BA000F79881217D2E531B4090050779009CE21
:1009CA00F82828730209E9020A3E020A0A020A12F0
:1009DA00020A16020A1E020A26020A2E020A367F94
:1009EA0001EF1218D9789BE6FC08E6FD7401936DB5
:1009FA007003E4936C70028F330FBF0FE4020AC1D5
:100A0A00789DE6F533020AE7789E800278A6E6F535
:100A1A0033020B0178A5E6F533020B2878AFE6F529
:100A2A0033020B4578B0E6F533020B6278B1E6F58E
:100A3A0033020B7FE53165326003020999A2173050
:100A4A009601B35013A296921730960C0531E531F0
:100A5A00C3940C4003E4F531A218309701B350D483
:100A6A00A29792183097CDE531B40C0050C6900A7F
:100A7A007FF8282873020AA3020ACF020AD5020ABB
:100A8A00F3020B07020B1A020B33020B50020B6D17
:100A9A00020B93020B99020B9F0533E533C3940FA4
:100AAA004003753301E5331218D9E493FF740193B7
:100ABA00789BCFF608EFF6E53375F004A424BDF968
:100ACA00740F020B88121333020A3E0533E533C34F
:100ADA0094034003E4F533789DA633E53375F004B7
:100AEA00A42417F97410020B881218E54003E4F5E0
:100AFA0033789EA633E5331218F4020B881218E5F0
:100B0A004003E4F53378A6A633E5331218F4806E71
:100B1A001218E54003E4F53378A5A633E53375F0FA
:100B2A0004A4242BF9741080550533E533C39404C7
:100B3A004003E4F53378AFA633E53375F004A42413
:100B4A0033F9741080380533E533C394034003E462
:100B5A00F53378B0A633E53375F004A42443F97469
:100B6A0010801B0533E533C394044003E4F533785E
:100B7A00B1A633E53375F004A4244FF9741035F0A7
:100B8A00FA7BFF1217D2020A3E121427020A3E12F9
:0B0B9A001835020A3E43A208020A3E82
:0A1B9B004552415300444F4E4500EF
:1019A000E4D3FCFD7B80FAF9F80206A6789BE6F505
:0D19B0005508E6F55622E56AAE6978062274
:10121400C215C216E4F532F533AE32AF331219A05B
:10122400401CE53164816016AF33AE3212180412EB
:101234001AA18F310533E53370DF053280DBE531E8
:10124400B48108E533153370021532AE32AF33E49E
:10125400C31219A2700CD215121B67E4F569F56A62
:10126400800785326985336AE4F56BF56C755480C3
:031274001219ACA0
:011277002254
:041804008F828E83BE
:101808001219A04027E582AE837806C333CE33CEC3
:10181800D8F9FD757102EE7879F6CFEDCFEF08F6BD
:0C1828007F50121A5F121BCFEF20E0F976
:011834002291
:031A2C00CDEFCD2E
:101A2F00757102EE7879F6ED08F67F50121A5F1293
:061A3F001BCFEF20E0F9CF
:011A4500227E
:101AA1007571017F501219F7121BCFEF20E0F97801
:031AB10079E6FFD4
:011AB400220F
:101A8C00121A2CE4FFFE0FBF00010EBE0FF8BFA010
:041A9C00F5121AA184
:011AA0002223
:06176A00CBEFCBCAEECA72
:10177000301503301627757103EA7879F6EB08F611
:1017800008EDF67F50121A5F121BCFEF20E0F9E44C
:0D179000FFFE0FBF00010EBE0FF8BFA0F559
:01179D002229
:1015C300753400753500753654E4F5331219B6C316
:1015D30033CE33CED8F97C002533FFEC3EFEAB345B
:1015E300AA35A93685338275830012051AFD1217B1
:1015F3006A0533E533C3940640D2756B00756C06F8
:0116030022C4
:101125008E318F321219B6C333CE33CED8F9256C32
:10113500FFE56B3EFEEEC0E0EFC0E0E531FDD0E03F
:10114500FFD0E0FE12176A056CE56C7002056B12A4
:1011550019B6C333CE33CED8F9256CFFE56B3EFE09
:10116500AD3212176A056CE56C7002056B0558E522
:101175005870020557C3E56C9440E56B9400401721
:10118500E4F56BF56C056AE56A70020569AE69FF01
:081195001219A05002D215222C
:10133300E4F56BF56C7BFF7A1B799B1217D2D216FF
:10134300E4F53EF53FAE3EAF3F1219A04021E53F25
:10135300AE3E7806C333CE33CED8F9F56C8E6B7DB3
:1013630081FF12176A053FE53F70DA053E80D6C25A
:10137300167BFF7A1B79A01217D2E4F569F56AF59B
:051383006BF56CC215C2
:011388002242
:1012DC00E4F53EF53FF540F541AE40AF411219A0A3
:1012EC004044E53F6481603EAF41AE4012180412A9
:1012FC001AA18F3FE53F64807022AF3E053EFCFD96
:10130C00FEFBFAF9120D517F2C120016AE40AF41C4
:10131C00E4FCFDFBFAF9120D51121BB80541E54135
:06132C0070B7054080B31C
:011332002298
:021470008F3EAD
:10147200E4F53FF540F541F542AE41AF421219A005
:101482004030E5406481602AAF42AE411218041236
:101492001AA18F40E540B4800FE53F653E7007AF6B
:1014A20042AE41021804053F0542E54270CB0541B8
:0214B20080C7F1
:0114B4002215
:101604001219AC78A6E6F559E4F557F5581215C346
:1016140085696D856A6E7F0112127830021A78A985
:10162400E6FE08E6FFE4FCFD7B64FAF9F812057BAC
:101634008F668E658D648C63300505C205121A763B
:011644002283
:1016FC00856931856A32E56C456B60080532E532E7
:10170C0070020531856D69856E6A1215C385316964
:10171C0085326AAE31AF321219A05007E4F569F583
:08172C006AD2157F0202127857
:101AB500740478FF769612FF0322740078FF7696F9
:041AC50012FF0322E7
:0300330002105F59
:0D105F00C0E0C0F0C083C082C0D075D008D2
:10106C00E5D954F8FF12071F10990810991010A811
:10107C001810C32010AA2810C33010C53810CB404C
:10108C0010C34810E4501101580000110F8574DA98
:10109C00C2DDC2DC7572007573008070800EE57164
:1010AC00700280560573E573700205721200268F6C
:1010BC00DAC2DDC2DC80558016D2DDC2DC804DC2C6
:1010CC00DDC2DCE5717004C2DA8041D2DA803DC247
:1010DC00DDD2DC756F048034AFDA121B8F0573E53B
:1010EC007370020572C2DDC2DCE5717004C2DA8075
:1010FC001BD2DA8017AFDA121B8FC2DDD2DC756F10
:0E110C00028009756F04C2DDC2DCD2DAC2DBDC
:0B111A00D0D0D082D083D0F0D0E032E3
:1018620043910C43920CE4F5DBEF25E0F5DB3017F6
:101872000343DB0175DD2575DC2575D84453F8FE7D
:0918820053F7FEE4F56FD2E822F1
:101A5F00E56F30E002FF22E4F570756F03EF25E0CC
:071A6F00F574D2DD7F0222B5
:1019F700E56F30E002FF22E4F5701571756F05EFB2
:0B1A070025E04401F574D2DD7F0222CF
:061BCF0020DBFDAF6F22D8
:0D0026001571AF70057074792FF8E6FF2298
:0C1B8F0074792570F8EFF60570157122CE
:0E1B5900E4F5847585FFF592F5A475A5FF22CD
:071BC100EE3395E0FDFC226C
:1018FE00C212C214C211D2A2C2A0C2A1E4FDFF1232
:10190E001982E4FD7F011219827F081212787F047A
:03191E000212783A
:10198200EF146011047016BD0104C2A78002D2A731
:0E199200A2A7921322BD0103C2A622D2A62252
:10127800EF14B40800505C90128D75F003A4C58378
:1012880025F0C583730212A50212AB0212B2021234
:10129800BE0212C00212BE0212CA0212D2D21275C5
:1012A800190122C212A21392A722D214751A057D1F
:1012B800017F010219828005C211C28722C211D2A0
:1012C8008722D211D28775180122C2A47F01121772
:0412D80034D2A42246
:10168400301212D5190F30A707C2A775191E80058D
:10169400D2A7751946E51AD39400400CD51A09C28D
:1016A40014E4FD7F01121982301111D5180E308710
:0D16B40006C28775180522D28775181E2200
:10194200C374039FFE1392A0EEA2E192A1AF80CFD7
:0F1952005480CFED547FCF4FCF8F80C2A2D2A24F
:011961002263
:0617D2008B408A418942B0
:1017D800E4FCCFECCF7D201219420CBC04F4E4FCED
:1017E800AB40AA41A9428C8275830012051AFD609C
:0B17F8000ACFECCF1219420CBC04E534
:0118030022C2
:04119D008F828E832C
:1011A100121BC1E47B0F7A27F9F8C31206A650037C
:1011B10090270FAF82AE83121BC17B197AFC79FF96
:1011C10078FFD31206A6400390FC19E4F531741B95
:1011D1002531F8E4F60531E531B405F2AE83AF828D
:1011E100121BC17B007A00791B120D51E51E701A8A
:1011F100753103741A2531F8E6FF741B2531F8C6E1
:10120100EFC6D531EE751B2080E27B007A00791B99
:031211000217D2EF
:1019BD0046554C4C0050524F47005A4C4F47004D26
:0D19CD004F440076322E34005472696700DA
:101B0500E6FE08E6FFE4FCFD2278CE1206E178C683
:031B15000206FACB
:03001300021921AE
:10192100C0E0C0D075D010200E0CAF8DEFAD8BF59F
:101931005EEDF55FD20E758D00758B00D0D0D0E0D5
:011941003273
:021734008F3FE5
:10173600E4F540F541C3E541953FE540940050236B
:10174600900000AF82AE83E4FCFD7B207A4EF9F870
:10175600D31206A64003A380EA0541E54170D605EB
:031766004080D2EE
:01176900225D
:0E1B67007BFF7A1979BD1217D27F0A0217345C
:0F1B3C00D20B301506121B67C20B2212160422A1
:05000E00C20B0216FC0C
:101A760078D212070600000000121B0E78CE12075D
:061A860006000000002232
:10003600121B59121BA51218FE7F041217342097A3
:10004600127BFF7A1979C21217D27F011214B5D228
:10005600AF80FE209612D2AF121A12C2177F70120C
:10006600186212121412097A7A1979C71204F6E480
:10007600FF1214B5D2AF121A127BFF7A1979CC127D
:1000860017D278B2E62430FD7F031219427F04129C
:1000960017347A1979D01204F6C2177F70121862D3
:1000A6007F01121734121214120019C21A1216C145
:1000B6007F01121734E4F560F56112001AA29692D8
:1000C60008A2979209E4F52478CA120706000000F0
:1000D60000E4F52578D2120706FFFFD8F178C6129C
:1000E600070600000000E4F55378CE12070600006C
:1000F6000000C20DC20BC20CE4F567F568F526F5E3
:1001060027F55EF55FC20EF562C20FF55DF55CF58B
:100116005BF55AF566F565F564F563F52078AFE6A7
:1001260024FE600B14600C2402700AD2018006D2F1
:10013600068002D20078B0E624FE6007047006D27C
:10014600028002D20778B1E624FE600B14600C240C
:1001560002700AD2038006D2048002D2053001174B
:10016600C20178A7121B057B64FAF9F812057B8F8A
:100176005D8E5C8D5B8C5A301AFDC21A300C33A230
:1001860008309601B3400BA209309701B340030231
:10019600026430961230970FC20CE4F567F5687F5B
:1001A60004121278E4F553A2969208A297920902D5
:1001B6000264209605209702D21030965630975347
:1001C600301031C21078C61206E1EC4D4E4F78D28F
:1001D600700C12070600000000121B0E801012079A
:1001E600060000000078C612070600000000D209CB
:1001F600D2088024789EE6601F0568E568700205CF
:1002060067D394B8E567940B400ED20C7F051212A3
:10021600788005E4F567F568A208309601B3501FAB
:10022600A2969208309618201015C201E553600771
:10023600E4F5537F0680057553017F07121278A2F5
:1002460009309701B35017A29792093097102010E2
:100256000DB20B300B05121B3C800312000E120769
:1002660045AF5DAE5CAD5BAC5AEC4D4E4F6026744F
:10027600FF2FF55DEE34FFF55CED34FFF55BEC34F6
:10028600FFF55AAF5DAE5CAD5BFC4D4E4F70062080
:100296000B03121B3CAF66AE65AD64AC63EC4D4E12
:1002A6004F602374FF2FF566EE34FFF565ED34FFDE
:1002B600F564EC34FFF563AF66AE65AD64FC4D4E98
:1002C6004F700312000E200E03020374C2AFC20E5B
:1002D600D2AFE4855F30855E2FF52EF52DAF30AEBB
:1002E6002FAD2EAC2D7B107A27F9F812057B8F30B7
:1002F6008E2F8D2E8C2DE4FB7A90F9F81214F98F3F
:10030600308E2F8D2E8C2D78A5E66009C374B89F8C
:10031600FF740B9EFEE56214601624FE6020240323
:100326007049C3EF94B0EE9404500E7562018009D3
:10033600D3EF9414EE940540357562038030C3EF15
:1003460094B0EE94045027756201300006200B032A
:10035600121B3C300305C203121A76300B02D20F71
:100366007BFF7A1979D51217D28003E4F562052549
:10037600E525C3940550030204F0E4F525FB7A0055
:10038600792812188B8E298F2AE5286402600302C9
:1003960004F078CA1206EDE8C0E0E9C0E0EAC0E081
:1003A600EBC0E0789DE6FDAF2AAE291213DBD0E064
:1003B600FBD0E0FAD0E0F9D0E0F8EB2FFFEA3EFE02
:1003C600E93DFDE83CFC78CA1206FA0524E524C39B
:1003D600940550030204F078CA1206E1E47B05FA9C
:1003E600F9F81214F978CA1206FA78CA1206E178F0
:1003F600C61206EDC3EF9BFFEE9AFEED99FDEC9853
:10040600FC78CA1206FA78D21206E178CA1206ED0C
:10041600D31206A6400A78CA1206E178D21206FA64
:10042600E553600A78D4E6FE08E68E2BF52C78CCE8
:10043600E6FE08E68E29F52AE5536006AF2CAE2BBC
:100446008004AF2AAE2912119D300B4E0527E527F1
:1004560070020526C3789C96E5261896403CE4F57E
:1004660026F5277F03121278300D0DE529FF1200BD
:1004760016AF2AE52A12001620151A78A6E6600C91
:10048600300F097F007E82121125C20FAF2AAE29D6
:100496001211258005121B67C20B78CA1206E17875
:1004A600CE1206FA78CA12070600000000E4F52408
:1004B600300405C204121A7630061678AB121B05F4
:1004C60078CE1206EDD31206A64006200B03121BA9
:1004D6003C30071678AD121B0578CE1206EDC31216
:1004E60006A65006300B0312000E12168402017D7A
:0B04F6007BFF1217D27F041217342284
:1018B300444C0021536967005A4C4F47004D4F4435
:1018C30000322E34004175672032342032303034F8
:0618D3000050524F4700D7
:10158000AF39AE38AD37AC36EC4D4E4F22EF24FFBD
:10159000F539EE34FFF538ED34FFF537EC34FFF56F
:1015A0003622E475392075384EF537F53622E47564
:1015B0003901F538F537F536227533007534007585
:0315C00035992238
:10074500121B75EF700302095A7F04121278E4F543
:1007550053C20CF567F5681219DAEF12071F093E47
:100765002409472A094A50089752078B61081963DB
:10077500086C6C087272086F73089B74090E760911
:1007850006780000095A7BFF7A1879B31217D2123E
:1007950015A2121B75EF700A121580600512158DD2
:1007A50080F0121580700302095A1219DA8F32127D
:1007B5001470E4F5391215B2E47F06FEFDFCAB3981
:1007C500AA38A937A836C31206BC501F121AA18F22
:1007D50032120016E5392401F539E43538F538E4E7
:1007E5003537F537E43536F53680CD121AA18F3217
:1007F500E53264806016E5326481601012001612DD
:100805001AA18F321200167531018003E4F531E526
:100815003170D8221215B91215AEF5321215806055
:10082500241215A2121B75EF700A121580600512AD
:10083500158D80F0121580600312095B0532E532D3
:10084500C3941A40D7121580601A7899B6AB070879
:10085500B6CD030209447BFF7A1879B61217D27F09
:100865000A021734020903B20D220212DC1215B96D
:10087500E4F532AB330535E535AA34700205341499
:10088500F9120501FF1200160532E532C3941A402C
:10089500E22243A2082275330075340075357712BC
:1008A50015AEF53212158060241215A2121B75EFD4
:1008B500700A121580600512158D80F01215806082
:1008C5000312095B0532E532C3940240D712158045
:1008D500602CAE77AF78EE3395E0FDFC78CE12064E
:1008E500EDC3EF9BF53DEE9AF53CED99F53BEC98A4
:1008F500F53AAF3D78A3E53CF608EFF680410215E1
:100905003D7F041212780213337A1879BB12096FEE
:100915007A1879C0121B1878B2E62430FF12001637
:10092500121BB87F761200167A1879C412096F7AED
:100935001879C8121B18021BB8E478A3F608F6024A
:1009450018350214277BFF7A1879D41217D27F0144
:050955001214B580FE44
:10095A00221219DAAB33AA34A9358532827583009B
:10096A00EF120559227BFF121B18121BB87BFF22BC
:0A1BA500E4F5955396BF53A27F228A
:1016C1005389F0438901538FFE758C70E4F58A5379
:1016D100B8FD53B7FDD2A9D28C53890F43899053DA
:1016E1008FEFF58DF58B4391105392EF53B8F7536C
:0B16F100B7F7D2ABD28ED28AD2AA2269
:03000B00021BAF26
:091BAF00D21A758C70758A00329F
:03001B00021BC8FD
:071BC800758D00758B0032E2
:101AC9000D0A003031323334353637383941424323
:041AD900444546003A
:101ADD00AF52AB46AA47A948055222AF45AE44AD19
:041AED0043AC4222A2
:1014B5005387BF75985053877FE4F5BABF0105433D
:1014C500A240800353A2BFE4F5BD75BE30F5BF75DC
:1014D500BD035391FE4392014391025392FDC21BFA
:1014E50053B8EF53B7EF43B81078C4F618F678C57C
:0414F500F6D2AC225D
:0300230002179E23
:10179E00C0E0C0D075D01030981E78C4E6C3940F48
:1017AE00501418E60624B3F8A69978C40618E6C3B2
:1017BE00941040027600C298309904C299C21BD090
:0417CE00D0D0E03265
:08000300201BFDD21B8F992286
:1019620078C4E6D39400401508E60624B3F8E6FFEF
:0F19720078C41608E6C394104005E4F6227F00FF
:011981002243
:03001600020003E2
:1019DA007F207E4E78C4E67010D3EF9400EE940018
:0C19EA004007EF1F70EE1E80EB12196228
:0119F60022CE
:101B1800120501FF600C120016740129F9E43AFA63
:031B280080EE222A
:0E1B750078C4E6D3940040037F01227F002253
:101A4600CEEFCEEE54F0C4540F901ACC93FF120092
:091A560016EE540F93FF02001676
:101B2B00CDEFCDCCEECCEEFF121A46CFEDCF021A95
:011B3B004663
:091BB8007BFF7A1A79C9021B189F
:0E0D51008F458E448D438C428B468A478948DD
:100D5F00E4F552EC4D4E4F7017E94A4B70057F305A
:100D6F00020016121ADD8F827583007430020E7422
:100D7F00121AEAEC33502AE5484547454670077F7B
:100D8F002D120016800D121ADD8F82758300742DBF
:100D9F00120559121AE81206988F458E448D438C0E
:100DAF0042755101754C00754BCA754A9A75493B8E
:100DBF00E4FFFEFDFCAB4CAA4BA94AA849D312068F
:100DCF00BC5003020E5F121AE8A8491206068F5094
:100DDF008E4F8D4E8C4DEC4D4E4F7004E551702360
:100DEF00E5502430FFE5484547454670051200168B
:100DFF00800EAE52121ADF8E82758300EF120559E4
:100E0F00E4F551AF4CAE4BAD4AAC49AB50AA4FA92C
:100E1F004EA84D12057BC8ECC8C9EDC9CAEECAC3AE
:100E2F00E5459FF545E5449AF544E54399F543E5D6
:100E3F004298F542AF4CAE4BAD4AAC49E47B0AFA4F
:100E4F00F9F81206068F4C8E4B8D4A8C49020DBF56
:100E5F00E547454845466010AB46AA47A948855225
:080E6F0082758300E4120559AD
:010E77002258
:100BA5000134C35001DBBF68028BBB800344B79897
:100BB5000407B3B004D5AFC805A9ABE00689A7F80B
:100BC5000775A410086DA02809719C400A819858E2
:100BD5000B9F94700CCA90880DE98CF90E048CA0BB
:100BE5000EA88AAC0F4D88B80FF786C410A184D023
:100BF500115182DC120580E812BB7EF413747D006E
:100C050014307B0C14F2791815B8772416807530DA
:100C1500174B733C1819714818ED6F5419C46D6062
:100C25001AA16B6C1B7E69781C6167841D4A6590EF
:100C35001E37639C1F2561A8201A5FB421125DC071
:100C4500220D5BCC230E59D8241557E4251F55F0EA
:100C5500262F53FC27425208285B501429764E2034
:100C65002A9B4C2C2BC04A382CEE48442E1E46504D
:100C75002F55445C308F426831D1407433173E8024
:100C850034633C8C35B13A98370938A4386636B0A8
:100C950039C734BC3B2D32C83C9D30D43E0F2EE0C5
:100CA5003F882CEC41062AF8428D29044418271068
:100CB50045AB251C4741232848E121344A861F407E
:100CC5004C311D4C4DE21B584F9C1964515D1770FA
:100CD5005323157C54EF138856C4119458A20FA0C2
:100CE5005A830DAC5C6D0BB85E6009C4605807D0C3
:100CF500625A05DC646203E8667301F4688A0000E1
:100D05006AA1FE0C6CB8FC186ECFFA2470E6F830B8
:100D150000000000000000000000000000000000CE
:100D250000000000000000000000000000000000BE
:100D350000000000000000000000000000000000AE
:0C0D4500000000000000000000000000A2
:1016450075F004E538A424A5F582E5F0340BF5839F
:10165500E49322FE740193FF75F004E538A422F5A6
:1016650083C37401939FFFE4939EFEE4228F398E1A
:0F167500388D378C36228F358E348D338C322260
:101AF100C3EF9DEE9C400AD3EF9BEE9A50037F010A
:041B0100227F00221D
:040E78008E368F37EC
:100E7C00E4F538121645FC740193FD12165D24A995
:100E8C00F582E5F0340BF583E493FA740193FBAF30
:100E9C0037AE36121AF1EF7003020F6812164512B4
:100EAC00165824A9F582E5F0340B1216648F3C8E8B
:100EBC003BF53AF53912165D24ABF582E5F0340BAF
:100ECC00F583E49312165824A7F582E5F0340B123F
:100EDC0016648F408E3FF53EF53DAD3EAC3D12069F
:100EEC00988F408E3F8D3E8C3DAE36AF37E4FCFD87
:100EFC00EEC0E0EFC0E0121645FE740193FBCAEEA3
:100F0C00CAD0E0FFD0E0FEC3EF9BFFEE9AFEED945B
:100F1C0000FDEC9400FCAB40AA3FA93EA83D120595
:100F2C007BAB3CAA3BA93AA8391214F9C8ECC8C946
:100F3C00EDC9CAEECACBEFCB12165D24A7F582E53C
:100F4C00F0340BF583E493FE740193FFE4FCFDEBAA
:100F5C002FFFEA3EFEED39FDEC38FC220538E53872
:0D0F6C00C3946A5003020E7FE4FFFEFDFCFB
:010F79002255
:01001A0022C3
:10138900121672AB39AA38A937A836E8C0E078A195
:10139900E6FE08E6FFE4FCFDD0E0F812057B121634
:1013A90072780E1206CD12167278A3E6FE08E6FFD1
:1013B900EE3395E0FDFCE5392FF539E5383EF53892
:1013C900E5373DF537E5363CF536AF39AE38AD375B
:0213D900FC22F4
:0213DB008D3152
:1013DD00120E7812167B12138912167BE5311460EA
:1013ED001C14702DE47FE87E03FDFCAB35AA34A9F7
:1013FD0033A83212057BE47BE87A0B800CAF35AE57
:10140D0034AD33AC32E47B03FAF9F81214F9121649
:09141D007BAF35AE34AD33AC32C7
:0114260022A3
:10050100BB010689828A83E0225002E722BBFE02F8
:09051100E32289828A83E493222B
:10051A00BB010CE58229F582E5833AF583E0225096
:10052A0006E92582F8E622BBFE06E92582F8E222E0
:0D053A00E58229F582E5833AF583E49322FA
:10054700BB010689828A83F0225002F722BBFE0193
:02055700F3228D
:10055900F8BB010DE58229F582E5833AF583E8F0D8
:10056900225006E92582C8F622BBFE05E92582C884
:02057900F2226C
:10057B00E88FF0A4CC8BF0A42CFCE98EF0A42CFC1F
:10058B008AF0EDA42CFCEA8EF0A4CDA8F08BF0A49D
:10059B002DCC3825F0FDE98FF0A42CCD35F0FCEBFC
:1005AB008EF0A4FEA9F0EB8FF0A4CFC5F02ECD39C1
:0F05BB00FEE43CFCEAA42DCE35F0FDE43CFC222E
:1005CA0075F008758200EF2FFFEE33FECD33CDCCE8
:1005DA0033CCC58233C5829BED9AEC99E58298406B
:1005EA000CF582EE9BFEED9AFDEC99FC0FD5F0D648
:1005FA00E4CEFBE4CDFAE4CCF9A88222B800C1B972
:10060A000059BA002DEC8BF084CFCECDFCE5F0CBAF
:10061A00F97818EF2FFFEE33FEED33FDEC33FCEBE8
:10062A0033FB10D703994004EB99FB0FD8E5E4F9A3
:10063A00FA227818EF2FFFEE33FEED33FDEC33FC90
:10064A00C933C910D7059BE99A4007EC9BFCE99A84
:10065A00F90FD8E0E4C9FAE4CCFB2275F010EF2FC9
:10066A00FFEE33FEED33FDCC33CCC833C810D707C9
:10067A009BEC9AE899400AED9BFDEC9AFCE899F804
:0E068A000FD5F0DAE4CDFBE4CCFAE4C8F92297
:1014F900C2D5E830E70FB2D5E4C39BFBE49AFAE41E
:1015090099F9E498F8EC30E717B2D512152F1206BD
:1015190006E4C39BFBE49AFAE499F9E498F880039A
:1015290012060630D50DE4C39FFFE49EFEE49DFD3F
:04153900E49CFC2210
:0E069800C3E49FFFE49EFEE49DFDE49CFC2273
:1006A600EB9FF5F0EA9E42F0E99D42F0EC6480C8CB
:0606B60064809845F0226B
:1006BC00EB9FF5F0EA9E42F0E99D42F0E89C45F094
:0106CC00220B
:1006CD00E86010ECA2E713FCED13FDEE13FEEF1343
:0406DD00FFD8F02230
:0C06E100E6FC08E6FD08E6FE08E6FF2245
:0D06ED00E6FB08E6F908E6FA08E6CBF8227D
:0C06FA00ECF608EDF608EEF608EFF6222C
:10070600D083D082E493F608740193F608740293BA
:09071600F608740393F6740473F1
:10071F00D083D082F8E4937012740193700DA3A369
:10072F0093F8740193F5828883E47374029368607D
:06073F00EFA3A3A380DF7D
:00000001FF
